:020000040000FA
:100000000000000000000000000000008316C9305E
:1000100085008312073099008501A401A301A30A7A
:100020004D28820700003D284128452849281430E2
:10003000A1000000A00B1928A10B19280034A41856
:100040005528A4140430230603195528A30A55285B
:10005000A4185528A4140430230603193128A30A30
:100060005528A301A30A5528A4185528A414013023
:10007000230603195528A3035528023085001720AD
:10008000003404308500172000341030850017201C
:100090000034203085001720003405185228851DB3
:1000A00034282828851D1F28A401230811204D2845
:0400B000FF2390009A
:02400E00D43F9D
:00000001FF
